 SwiQdl

 Timestamp is 54003939 (Fri Aug 29 16:26:33 2014)

 Preferred load address is 10000000

 Start         Length     Name                   Class
 0001:00000000 00003830H .text                   CODE
 0002:00000000 0000248eH .rdata                  DATA
 0002:00002490 0000000cH .xdata                  DATA
 0002:0000249c 00000014H .idata$2                DATA
 0002:000024b0 00000014H .idata$3                DATA
 0002:000024c4 0000008cH .idata$4                DATA
 0002:00002550 0000000cH .idata$6                DATA
 0002:00002560 0000006aH .edata                  DATA
 0003:00000000 0000008cH .idata$5                DATA
 0003:0000008c 00000004H .CRT$XCA                DATA
 0003:00000090 00000004H .CRT$XCAA               DATA
 0003:00000094 00000004H .CRT$XCZ                DATA
 0003:00000098 00000004H .CRT$XIA                DATA
 0003:0000009c 00000004H .CRT$XIZ                DATA
 0003:000000a0 00000004H .CRT$XPA                DATA
 0003:000000a4 00000004H .CRT$XPZ                DATA
 0003:000000a8 00000004H .CRT$XTA                DATA
 0003:000000ac 00000004H .CRT$XTZ                DATA
 0003:000000b0 00000210H .data                   DATA
 0003:000002c0 00000364H .bss                    DATA
 0004:00000000 000000f0H .pdata                  DATA
 0005:00000000 00000058H .rsrc$01                DATA
 0005:00000060 0000040cH .rsrc$02                DATA

  Address         Publics by Value              Rva+Base       Lib:Object

 0000:00000000       ___safe_se_handler_count   00000000     <absolute>
 0000:00000000       ___safe_se_handler_table   00000000     <absolute>
 0001:00000000       CalculateCRC16             10001000 f   crc.obj
 0001:00000040       ?DisplayMemoryStatus@@YAXXZ 10001040 f   swiusb.obj
 0001:0000008c       ?OpenOutModemBulkPipe11@@YAPAXU_USB_ENDPOINT_DESCRIPTOR@@@Z 1000108c f   swiusb.obj
 0001:0000011c       ?OpenInModemBulkPipe10@@YAPAXU_USB_ENDPOINT_DESCRIPTOR@@@Z 1000111c f   swiusb.obj
 0001:000001ac       ?GetChannel@@YAPAU_SW_CHANNEL@@PAU1@K@Z 100011ac f   swiusb.obj
 0001:000001f4       ?SWIWriteCompletionRoutine@@YAKPAX@Z 100011f4 f   swiusb.obj
 0001:000001f4       ?SWIReadCompletionRoutine@@YAKPAX@Z 100011f4 f   swiusb.obj
 0001:00000598       ?BulkOutThread@@YAXPAPAX@Z 10001598 f   swiusb.obj
 0001:000007e0       ?USBDeviceNotifications@@YAHPAXKPAPAK111@Z 100017e0 f   swiusb.obj
 0001:00000e48       USBInstallDriver           10001e48 f   swiusb.obj
 0001:00000e6c       ?VerifyPacket@@YAHPAEK@Z   10001e6c f   swiusb.obj
 0001:00000ec8       ?HandleErrorResponse@@YAXXZ 10001ec8 f   swiusb.obj
 0001:00000f70       ?ProcessPacket@@YAXPAU_SW_CHANNEL@@PAEI@Z 10001f70 f   swiusb.obj
 0001:00001208       ?SendData@@YAHPAU_SW_CHANNEL@@@Z 10002208 f   swiusb.obj
 0001:0000150c       ?ValidateData@@YAKPAU_SW_CHANNEL@@PAXK@Z 1000250c f   swiusb.obj
 0001:00001600       ?BuildPacket@@YAHPAU_SW_CHANNEL@@@Z 10002600 f   swiusb.obj
 0001:0000190c       ?StateMachineThread@@YAKPAX@Z 1000290c f   swiusb.obj
 0001:00001a84       ?GetFWFile@@YAHAAU_GOBI_FW@@@Z 10002a84 f   swiusb.obj
 0001:00001b74       ?GetGobiFirmware@@YAHXZ    10002b74 f   swiusb.obj
 0001:00001fd0       ?BulkInThread@@YAXPAPAX@Z  10002fd0 f   swiusb.obj
 0001:000025e0       USBDeviceAttach            100035e0 f   swiusb.obj
 0001:000032c4       EventModify                100042c4 f   coredll:COREDLL.dll
 0001:000032d4       NKDbgPrintfW               100042d4 f   coredll:COREDLL.dll
 0001:000032e4       GlobalMemoryStatus         100042e4 f   coredll:COREDLL.dll
 0001:000032f4       GetLastError               100042f4 f   coredll:COREDLL.dll
 0001:00003304       WaitForMultipleObjects     10004304 f   coredll:COREDLL.dll
 0001:00003314       GetTickCount               10004314 f   coredll:COREDLL.dll
 0001:00003324       WaitForSingleObject        10004324 f   coredll:COREDLL.dll
 0001:00003334       LocalFree                  10004334 f   coredll:COREDLL.dll
 0001:00003344       VirtualFree                10004344 f   coredll:COREDLL.dll
 0001:00003354       TerminateThread            10004354 f   coredll:COREDLL.dll
 0001:00003364       CloseHandle                10004364 f   coredll:COREDLL.dll
 0001:00003374       Sleep                      10004374 f   coredll:COREDLL.dll
 0001:00003384       ReadFile                   10004384 f   coredll:COREDLL.dll
 0001:00003394       SetFilePointer             10004394 f   coredll:COREDLL.dll
 0001:000033a4       memcpy                     100043a4 f   coredll:COREDLL.dll
 0001:000033b4       memset                     100043b4 f   coredll:COREDLL.dll
 0001:000033c4       GetFileSize                100043c4 f   coredll:COREDLL.dll
 0001:000033d4       CreateFileW                100043d4 f   coredll:COREDLL.dll
 0001:000033e4       swprintf                   100043e4 f   coredll:COREDLL.dll
 0001:000033f4       RegCloseKey                100043f4 f   coredll:COREDLL.dll
 0001:00003404       _wcslwr                    10004404 f   coredll:COREDLL.dll
 0001:00003414       RegQueryValueExW           10004414 f   coredll:COREDLL.dll
 0001:00003424       RegOpenKeyExW              10004424 f   coredll:COREDLL.dll
 0001:00003434       wcscmp                     10004434 f   coredll:COREDLL.dll
 0001:00003444       VirtualAlloc               10004444 f   coredll:COREDLL.dll
 0001:00003454       CeSetThreadPriority        10004454 f   coredll:COREDLL.dll
 0001:00003464       CreateThread               10004464 f   coredll:COREDLL.dll
 0001:00003474       LocalAlloc                 10004474 f   coredll:COREDLL.dll
 0001:00003484       CreateEventW               10004484 f   coredll:COREDLL.dll
 0001:00003494       MultiByteToWideChar        10004494 f   coredll:COREDLL.dll
 0001:000034a4       _DllMainCRTStartup         100044a4 f   corelibc:pegdmain.obj
 0001:0000353c       __security_check_cookie    1000453c     corelibc:armsecgs.obj
 0001:00003550       __gsfailure                10004550     corelibc:armsecgs.obj
 0001:00003594       _cinit                     10004594 f   corelibc:crt0dat.obj
 0001:00003704       _cexit                     10004704 f   corelibc:crt0dat.obj
 0001:00003720       DllMain                    10004720 f   corelibc:dllmain.obj
 0001:00003738       __security_init_cookie     10004738 f   corelibc:seccinit.obj
 0001:00003788       __GSHandlerCheckCommon     10004788 f   LIBCMT:gshandler.obj
 0001:000037d0       __GSHandlerCheck           100047d0 f   LIBCMT:gshandler.obj
 0001:00003800       __report_gsfailure         10004800 f   coredll:COREDLL.dll
 0001:00003810       DisableThreadLibraryCalls  10004810 f   coredll:COREDLL.dll
 0001:00003820       __security_gen_cookie      10004820 f   coredll:COREDLL.dll
 0002:00000000       ??_C@_1DI@FLOGFLCI@?$AAS?$AAW?$AAI?$AAQ?$AAD?$AAL?$AA?5?$AAD?$AAi?$AAs?$AAp?$AAl?$AAa?$AAy?$AAM?$AAe?$AAm?$AAo?$AAr?$AAy?$AAS?$AAt?$AAa?$AAt?$AAu?$AAs?$AA?3?$AA?$AA@ 10005000     swiusb.obj
 0002:00000038       ??_C@_1KE@LBNPNIMH@?$AA?$CF?$AAs?$AA?5?$AAM?$AAe?$AAm?$AA?5?$AAs?$AAt?$AAa?$AAt?$AAu?$AAs?$AA?3?$AA?5?$AAT?$AAo?$AAt?$AAa?$AAl?$AAP?$AAh?$AAy?$AAs?$AA?3?$AA?5?$AA?$CF?$AAd?$AA?0?$AA?5?$AAA?$AAv@ 10005038     swiusb.obj
 0002:000000dc       ??_C@_1DO@FCJAHJLB@?$AAS?$AAW?$AAI?$AAQ?$AAD?$AAL?$AA?5?$AAO?$AAp?$AAe?$AAn?$AAO?$AAu?$AAt?$AAM?$AAo?$AAd?$AAe?$AAm?$AAB?$AAu?$AAl?$AAk?$AAP?$AAi?$AAp?$AAe?$AA1?$AA1?$AA?3?$AA?$AA@ 100050dc     swiusb.obj
 0002:00000120       ??_C@_1GK@CANBIIKH@?$AA?$CF?$AAs?$AA?5?$AAF?$AAa?$AAi?$AAl?$AAe?$AAd?$AA?5?$AAt?$AAo?$AA?5?$AAo?$AAp?$AAe?$AAn?$AA?5?$AAE?$AAn?$AAd?$AAP?$AAo?$AAi?$AAn?$AAt?$AA?5?$AA?$CD?$AA?$CF?$AAd?$AA?5?$AAo@ 10005120     swiusb.obj
 0002:0000018c       ??_C@_1DM@LODENNIM@?$AAS?$AAW?$AAI?$AAQ?$AAD?$AAL?$AA?5?$AAO?$AAp?$AAe?$AAn?$AAI?$AAn?$AAM?$AAo?$AAd?$AAe?$AAm?$AAB?$AAu?$AAl?$AAk?$AAP?$AAi?$AAp?$AAe?$AA1?$AA0?$AA?3?$AA?$AA@ 1000518c     swiusb.obj
 0002:000001c8       ??_C@_1GI@DDDHJAGF@?$AA?$CF?$AAs?$AA?5?$AAF?$AAa?$AAi?$AAl?$AAe?$AAd?$AA?5?$AAt?$AAo?$AA?5?$AAo?$AAp?$AAe?$AAn?$AA?5?$AAE?$AAn?$AAd?$AAP?$AAo?$AAi?$AAn?$AAt?$AA?5?$AA?$CD?$AA?$CF?$AAd?$AA?5?$AAi@ 100051c8     swiusb.obj
 0002:00000230       ??_C@_1FA@DCDCBIMM@?$AA?$CF?$AAs?$AA?5?$AAI?$AAs?$AAs?$AAu?$AAe?$AA?5?$AAt?$AAr?$AAa?$AAn?$AAs?$AAf?$AAe?$AAr?$AA?5?$AAf?$AAa?$AAi?$AAl?$AAe?$AAd?$AA?5?$AAa?$AAt?$AA?5?$AAe?$AAr?$AAr?$AAo@ 10005230     swiusb.obj
 0002:00000280       ??_C@_1CO@JPBBAIFD@?$AA?$CF?$AAs?$AA?5?$AAT?$AAr?$AAa?$AAn?$AAs?$AAf?$AAe?$AAr?$AA?5?$AAa?$AAb?$AAo?$AAr?$AAt?$AAe?$AAd?$AA?4?$AA?$AN?$AA?6?$AA?$AA@ 10005280     swiusb.obj
 0002:000002b0       ??_C@_1GM@JNIOBDFN@?$AA?$CF?$AAs?$AA?5?$AAA?$AAb?$AAo?$AAr?$AAt?$AA?5?$AAt?$AAr?$AAa?$AAn?$AAs?$AAf?$AAe?$AAr?$AA?5?$AAf?$AAa?$AAi?$AAl?$AAe?$AAd?$AA?0?$AA?5?$AAa?$AAn?$AAd?$AA?5?$AAt?$AAr@ 100052b0     swiusb.obj
 0002:00000320       ??_C@_1IE@LCPMOLEF@?$AA?$CF?$AAs?$AA?5?$AAA?$AAb?$AAo?$AAr?$AAt?$AA?5?$AAt?$AAr?$AAa?$AAn?$AAs?$AAf?$AAe?$AAr?$AA?5?$AAf?$AAa?$AAi?$AAl?$AAe?$AAd?$AA?0?$AA?5?$AAb?$AAu?$AAt?$AA?5?$AAt?$AAr@ 10005320     swiusb.obj
 0002:000003a8       ??_C@_1JC@OELNJEEL@?$AA?$CF?$AAs?$AA?5?$AAA?$AAb?$AAo?$AAr?$AAt?$AA?5?$AAt?$AAr?$AAa?$AAn?$AAs?$AAf?$AAe?$AAr?$AA?5?$AAf?$AAa?$AAi?$AAl?$AAe?$AAd?$AA?0?$AA?5?$AAb?$AAu?$AAt?$AA?5?$AAt?$AAr@ 100053a8     swiusb.obj
 0002:0000043c       ??_C@_1CM@MPHFDBCD@?$AAS?$AAW?$AAI?$AAQ?$AAD?$AAL?$AA?5?$AAT?$AAr?$AAa?$AAn?$AAs?$AAm?$AAi?$AAt?$AAB?$AAy?$AAt?$AAe?$AAs?$AA?3?$AA?$AA@ 1000543c     swiusb.obj
 0002:00000468       ??_C@_1FA@KCAIDLB@?$AA?$CK?$AA?$CK?$AA?$CK?$AA?$CF?$AAs?$AA?5?$AAT?$AAr?$AAa?$AAn?$AAs?$AAf?$AAe?$AAr?$AA?5?$AAs?$AAt?$AAa?$AAt?$AAu?$AAs?$AA?5?$AAe?$AAr?$AAr?$AAo?$AAr?$AA?5?$AA?$DN?$AA?5?$AA?$CF?$AA0@ 10005468     swiusb.obj
 0002:000004b8       ??_C@_1EO@JLCNGLJO@?$AA?$CF?$AAs?$AA?5?$AAC?$AAh?$AAa?$AAn?$AAn?$AAe?$AAl?$AA?5?$AA?$CD?$AA?$CF?$AAd?$AA?5?$AAe?$AAx?$AAi?$AAt?$AAs?$AA?0?$AA?5?$AAt?$AAi?$AAc?$AAk?$AAC?$AAo?$AAu?$AAn?$AAt?$AA?5@ 100054b8     swiusb.obj
 0002:00000508       ??_C@_1GG@PLLBCCPF@?$AA?$CF?$AAs?$AA?5?$AAT?$AAh?$AAr?$AAe?$AAa?$AAd?$AA?5?$AAe?$AAx?$AAi?$AAt?$AAs?$AA?5?$AAb?$AAe?$AAc?$AAa?$AAu?$AAs?$AAe?$AA?5?$AAh?$AAD?$AAe?$AAv?$AAi?$AAc?$AAe?$AAC@ 10005508     swiusb.obj
 0002:00000570       ??_C@_1CI@PJGCKFCO@?$AA?$CF?$AAs?$AA?5?$AAU?$AAS?$AAB?$AA?5?$AAD?$AAe?$AAv?$AAi?$AAc?$AAe?$AA?5?$AAO?$AAu?$AAt?$AA?$AN?$AA?6?$AA?$AA@ 10005570     swiusb.obj
 0002:00000598       ??_C@_1CM@NMFHKBG@?$AAS?$AAW?$AAI?$AAQ?$AAD?$AAL?$AA?5?$AAB?$AAu?$AAl?$AAk?$AAO?$AAu?$AAt?$AAT?$AAh?$AAr?$AAe?$AAa?$AAd?$AA?3?$AA?$AA@ 10005598     swiusb.obj
 0002:000005c8       ??_C@_1MA@LCJAMCJG@?$AA?$CF?$AAs?$AA?5?$AAT?$AAh?$AAr?$AAe?$AAa?$AAd?$AA?5?$AAw?$AAa?$AAi?$AAt?$AAs?$AA?5?$AAf?$AAo?$AAr?$AA?5?$AAm?$AAu?$AAl?$AAt?$AAi?$AAp?$AAl?$AAe?$AA?5?$AAo?$AAu?$AAt@ 100055c8     swiusb.obj
 0002:00000688       ??_C@_1DM@LKGCAIJN@?$AA?$CF?$AAs?$AA?5?$AAD?$AAe?$AAv?$AAi?$AAc?$AAe?$AA?5?$AAR?$AAe?$AAm?$AAo?$AAv?$AAe?$AAd?$AA?5?$AA?$EA?$AA?5?$AAt?$AAc?$AA?5?$AA?$DN?$AA?5?$AA?$CF?$AAd?$AA?$AN?$AA?6?$AA?$AA@ 10005688     swiusb.obj
 0002:000006c8       ??_C@_1EI@IHOJFPCE@?$AA?$CF?$AAs?$AA?5?$AAF?$AAa?$AAi?$AAl?$AAe?$AAd?$AA?5?$AAt?$AAo?$AA?5?$AAf?$AAr?$AAe?$AAe?$AA?5?$AAm?$AAe?$AAm?$AAo?$AAr?$AAy?$AA?5?$AAa?$AAt?$AA?5?$AA0?$AAx?$AA?$CF?$AAx@ 100056c8     swiusb.obj
 0002:00000710       ??_C@_1DK@FHMDCEKO@?$AAp?$AAC?$AAh?$AAa?$AAn?$AAn?$AAe?$AAl?$AA?9?$AA?$DO?$AAm?$AA_?$AAp?$AAB?$AAu?$AAf?$AAf?$AAe?$AAr?$AA?5?$AAf?$AAr?$AAe?$AAe?$AAd?$AA?4?$AA?$AN?$AA?6?$AA?$AA@ 10005710     swiusb.obj
 0002:00000750       ??_C@_1EO@GFOMOPIB@?$AA?$CF?$AAs?$AA?5?$AAb?$AAu?$AAl?$AAk?$AA?5?$AAo?$AAu?$AAt?$AA?5?$AAc?$AAh?$AAa?$AAn?$AAn?$AAe?$AAl?$AA?5?$AA?$CF?$AAd?$AA?5?$AAe?$AAx?$AAi?$AAt?$AAs?$AA?5?$AAt?$AAi?$AAm@ 10005750     swiusb.obj
 0002:000007a0       ??_C@_1EM@EABFJCBK@?$AA?$CF?$AAs?$AA?5?$AAb?$AAu?$AAl?$AAk?$AA?5?$AAi?$AAn?$AA?5?$AAc?$AAh?$AAa?$AAn?$AAn?$AAe?$AAl?$AA?5?$AA?$CF?$AAd?$AA?5?$AAe?$AAx?$AAi?$AAt?$AAs?$AA?5?$AAt?$AAi?$AAm?$AAe@ 100057a0     swiusb.obj
 0002:000007ec       ??_C@_1DM@FOGNJNCJ@?$AAS?$AAt?$AAa?$AAt?$AAe?$AA?5?$AAm?$AAa?$AAc?$AAh?$AAi?$AAn?$AAe?$AA?5?$AAe?$AAx?$AAi?$AAt?$AAs?$AA?5?$AAt?$AAi?$AAm?$AAe?$AAo?$AAu?$AAt?$AA?$AN?$AA?6?$AA?$AA@ 100057ec     swiusb.obj
 0002:00000828       ??_C@_1DK@EIKMDAGF@?$AA?$CF?$AAs?$AA?5?$AAD?$AAe?$AAv?$AAi?$AAc?$AAe?$AA?5?$AAr?$AAe?$AAm?$AAo?$AAv?$AAe?$AAd?$AA?4?$AA?5?$AAt?$AAc?$AA?5?$AA?$DN?$AA?5?$AA?$CF?$AAd?$AA?$AN?$AA?6?$AA?$AA@ 10005828     swiusb.obj
 0002:00000864       ??_C@_1DO@IPLDCPHH@?$AAS?$AAW?$AAI?$AAQ?$AAD?$AAL?$AA?5?$AAU?$AAS?$AAB?$AAD?$AAe?$AAv?$AAi?$AAc?$AAe?$AAN?$AAo?$AAt?$AAi?$AAf?$AAi?$AAc?$AAa?$AAt?$AAi?$AAo?$AAn?$AAs?$AA?3?$AA?$AA@ 10005864     swiusb.obj
 0002:000008a8       ??_C@_1FI@NDHDIDPF@?$AA?$CF?$AAs?$AA?5?$AAU?$AAn?$AAh?$AAa?$AAn?$AAd?$AAl?$AAe?$AAd?$AA?5?$AAU?$AAS?$AAB?$AA?5?$AAn?$AAo?$AAt?$AAi?$AAf?$AAi?$AAc?$AAa?$AAt?$AAi?$AAo?$AAn?$AA?5?$AAd?$AAw@ 100058a8     swiusb.obj
 0002:00000900       ??_C@_1DC@OIEKEGCI@?$AAS?$AAW?$AAI?$AAQ?$AAD?$AAL?$AA?5?$AAU?$AAS?$AAB?$AAI?$AAn?$AAs?$AAt?$AAa?$AAl?$AAl?$AAD?$AAr?$AAi?$AAv?$AAe?$AAr?$AA?3?$AA?$AA@ 10005900     swiusb.obj
 0002:00000934       ??_C@_1DE@FIGCKAOO@?$AA?$CF?$AAs?$AA?5?$AAC?$AAa?$AAl?$AAl?$AAe?$AAd?$AA?5?$AAf?$AAo?$AAr?$AA?5?$AAd?$AAr?$AAi?$AAv?$AAe?$AAr?$AA?5?$AA?$CF?$AAs?$AA?$AN?$AA?6?$AA?$AA@ 10005934     swiusb.obj
 0002:00000968       ??_C@_1CK@BGKNJLBI@?$AAS?$AAW?$AAI?$AAQ?$AAD?$AAL?$AA?5?$AAV?$AAe?$AAr?$AAi?$AAf?$AAy?$AAP?$AAa?$AAc?$AAk?$AAe?$AAt?$AA?3?$AA?$AA@ 10005968     swiusb.obj
 0002:00000998       ??_C@_1GO@ILGONHHE@?$AA?$CF?$AAs?$AA?5?$AAP?$AAa?$AAc?$AAk?$AAe?$AAt?$AA?5?$AAC?$AAR?$AAC?$AA?5?$AAv?$AAe?$AAr?$AAi?$AAf?$AAi?$AAc?$AAa?$AAt?$AAi?$AAo?$AAn?$AA?5?$AAf?$AAa?$AAi?$AAl?$AAu@ 10005998     swiusb.obj
 0002:00000a08       ??_C@_1FG@PMOBALIE@?$AA?$CF?$AAs?$AA?5?$AAS?$AAi?$AAg?$AAn?$AAa?$AAl?$AA?5?$AAs?$AAh?$AAu?$AAt?$AA?5?$AAd?$AAo?$AAw?$AAm?$AA?5?$AAm?$AAo?$AAd?$AAe?$AAm?$AA?5?$AAe?$AAv?$AAe?$AAn?$AAt?$AA?4@ 10005a08     swiusb.obj
 0002:00000a60       ??_C@_1JA@BAALDGPM@?$AA?$CF?$AAs?$AA?5?$AAN?$AAo?$AA?5?$AAm?$AAo?$AAr?$AAe?$AA?5?$AAf?$AAi?$AAr?$AAm?$AAw?$AAa?$AAr?$AAe?$AA?5?$AAd?$AAo?$AAw?$AAn?$AAl?$AAo?$AAa?$AAd?$AA?5?$AAr?$AAe?$AAt@ 10005a60     swiusb.obj
 0002:00000af0       ??_C@_1DI@NNHDLNNF@?$AAS?$AAW?$AAI?$AAQ?$AAD?$AAL?$AA?5?$AAH?$AAa?$AAn?$AAd?$AAl?$AAe?$AAE?$AAr?$AAr?$AAo?$AAr?$AAR?$AAe?$AAs?$AAp?$AAo?$AAn?$AAs?$AAe?$AA?3?$AA?$AA@ 10005af0     swiusb.obj
 0002:00000b28       ??_C@_1EE@MEFLHPPJ@?$AA?$CF?$AAs?$AA?5?$AAF?$AAi?$AAr?$AAm?$AAw?$AAa?$AAr?$AAe?$AA?5?$AAd?$AAo?$AAw?$AAn?$AAl?$AAo?$AAa?$AAd?$AA?5?$AAr?$AAe?$AAt?$AAr?$AAy?$AA?5?$AA?$CD?$AA?$CF?$AAd?$AA?4?$AA?$AN@ 10005b28     swiusb.obj
 0002:00000b6c       ??_C@_1DK@KPMPLFCG@?$AA?$CF?$AAs?$AA?5?$AAB?$AAa?$AAd?$AA?5?$AAC?$AAR?$AAC?$AA?5?$AAe?$AAr?$AAr?$AAo?$AAr?$AA?5?$AAr?$AAe?$AAc?$AAe?$AAi?$AAv?$AAe?$AAd?$AA?4?$AA?$AN?$AA?6?$AA?$AA@ 10005b6c     swiusb.obj
 0002:00000ba8       ??_C@_1EI@HHDMIJAL@?$AA?$CF?$AAs?$AA?5?$AAI?$AAn?$AAv?$AAa?$AAl?$AAi?$AAd?$AA?5?$AAl?$AAe?$AAn?$AAg?$AAt?$AAh?$AA?5?$AAe?$AAr?$AAr?$AAo?$AAr?$AA?5?$AAr?$AAe?$AAc?$AAe?$AAi?$AAv?$AAe?$AAd@ 10005ba8     swiusb.obj
 0002:00000bf0       ??_C@_1IM@FCHFBBEN@?$AA?$CF?$AAs?$AA?5?$AAT?$AAa?$AAr?$AAg?$AAe?$AAt?$AA?5?$AAt?$AAi?$AAm?$AAe?$AA?5?$AAo?$AAu?$AAt?$AA?5?$AAe?$AAr?$AAr?$AAo?$AAr?$AA?5?$AAr?$AAe?$AAc?$AAe?$AAi?$AAv?$AAe@ 10005bf0     swiusb.obj
 0002:00000c80       ??_C@_1HE@PBFHEHEE@?$AA?$CF?$AAs?$AA?5?$AAd?$AAo?$AAn?$AAe?$AA?5?$AAr?$AAe?$AAs?$AAp?$AAo?$AAn?$AAs?$AAe?$AA?5?$AAe?$AAr?$AAr?$AAo?$AAr?$AA?3?$AA?5?$AA?$CF?$AAx?$AA?0?$AA?5?$AAi?$AAm?$AAa?$AAg@ 10005c80     swiusb.obj
 0002:00000cf8       ??_C@_1HE@LOLDGAEG@?$AA?$CF?$AAs?$AA?5?$AAW?$AAr?$AAi?$AAt?$AAe?$AA?5?$AAr?$AAe?$AAs?$AAp?$AAo?$AAn?$AAs?$AAe?$AA?5?$AAd?$AAo?$AAe?$AAs?$AAn?$AA?8?$AAt?$AA?5?$AAm?$AAa?$AAt?$AAc?$AAh?$AA?5@ 10005cf8     swiusb.obj
 0002:00000d70       ??_C@_1HC@GNBPPBOB@?$AA?$CF?$AAs?$AA?5?$AAO?$AAp?$AAe?$AAn?$AA?5?$AAr?$AAe?$AAs?$AAp?$AAo?$AAn?$AAs?$AAe?$AA?5?$AAd?$AAo?$AAe?$AAn?$AAs?$AA?8?$AAt?$AA?5?$AAm?$AAa?$AAt?$AAc?$AAh?$AA?5?$AAt@ 10005d70     swiusb.obj
 0002:00000de8       ??_C@_1GC@OOKECEPF@?$AA?$CF?$AAs?$AA?5?$AAO?$AAp?$AAe?$AAn?$AA?5?$AAU?$AAQ?$AAC?$AAN?$AA?5?$AAr?$AAe?$AAs?$AAp?$AAo?$AAn?$AAs?$AAe?$AA?5?$AAe?$AAr?$AAr?$AAo?$AAr?$AA?5?$AAr?$AAe?$AAc?$AAe@ 10005de8     swiusb.obj
 0002:00000e50       ??_C@_1EI@PMCEPIOA@?$AA?$CF?$AAs?$AA?5?$AAn?$AAo?$AA?5?$AAn?$AAe?$AAe?$AAd?$AA?5?$AAt?$AAo?$AA?5?$AAd?$AAo?$AAw?$AAn?$AAl?$AAo?$AAa?$AAd?$AA?5?$AAU?$AAQ?$AAC?$AAN?$AA?5?$AAf?$AAi?$AAl?$AAe@ 10005e50     swiusb.obj
 0002:00000e98       ??_C@_1GC@PFFICNNC@?$AA?$CF?$AAs?$AA?5?$AAO?$AAp?$AAe?$AAn?$AA?5?$AAA?$AAM?$AAS?$AAS?$AA?5?$AAr?$AAe?$AAs?$AAp?$AAo?$AAn?$AAs?$AAe?$AA?5?$AAe?$AAr?$AAr?$AAo?$AAr?$AA?5?$AAr?$AAe?$AAc?$AAe@ 10005e98     swiusb.obj
 0002:00000f00       ??_C@_1EI@CPPLALLM@?$AA?$CF?$AAs?$AA?5?$AAN?$AAo?$AA?5?$AAn?$AAe?$AAe?$AAd?$AA?5?$AAt?$AAo?$AA?5?$AAd?$AAo?$AAw?$AAn?$AAl?$AAo?$AAa?$AAd?$AA?5?$AAa?$AAm?$AAs?$AAs?$AA?5?$AAf?$AAi?$AAl?$AAe@ 10005f00     swiusb.obj
 0002:00000f48       ??_C@_1CM@CPLFGGGF@?$AAS?$AAW?$AAI?$AAQ?$AAD?$AAL?$AA?5?$AAP?$AAr?$AAo?$AAc?$AAe?$AAs?$AAs?$AAP?$AAa?$AAc?$AAk?$AAe?$AAt?$AA?3?$AA?$AA@ 10005f48     swiusb.obj
 0002:00000f78       ??_C@_1HE@OOGALAIL@?$AA?$CF?$AAs?$AA?5?$AAH?$AAe?$AAl?$AAl?$AAo?$AA?5?$AAr?$AAe?$AAs?$AAp?$AAo?$AAn?$AAs?$AAe?$AA?5?$AAd?$AAo?$AAe?$AAn?$AAs?$AA?8?$AAt?$AA?5?$AAm?$AAa?$AAt?$AAc?$AAh?$AA?5@ 10005f78     swiusb.obj
 0002:00000ff0       ??_C@_1EA@OAJFBDIN@?$AA?$CF?$AAs?$AA?5?$AAS?$AAe?$AAn?$AAd?$AA?5?$AAd?$AAa?$AAt?$AAa?$AA?5?$AAa?$AAb?$AAo?$AAr?$AAt?$AAe?$AAd?$AA?4?$AA?5?$AAt?$AAc?$AA?5?$AA?$DN?$AA?5?$AA?$CF?$AAd?$AA?$AN?$AA?6?$AA?$AA@ 10005ff0     swiusb.obj
 0002:00001030       ??_C@_1EK@DHAPCNJA@?$AA?$CF?$AAs?$AA?5?$AAD?$AAe?$AAv?$AAi?$AAc?$AAe?$AA?5?$AAi?$AAs?$AA?5?$AAo?$AAu?$AAt?$AA?5?$AAd?$AAu?$AAr?$AAi?$AAn?$AAg?$AA?5?$AAs?$AAe?$AAn?$AAd?$AA?5?$AAd?$AAa?$AAt@ 10006030     swiusb.obj
 0002:00001080       ??_C@_1HM@DENJEOMN@?$AA?$CF?$AAs?$AA?5?$AAF?$AAa?$AAi?$AAl?$AAe?$AAd?$AA?5?$AAt?$AAo?$AA?5?$AAr?$AAe?$AAa?$AAd?$AA?5?$AAd?$AAa?$AAt?$AAa?$AA?5?$AAf?$AAr?$AAo?$AAm?$AA?5?$AA?$CF?$AAs?$AA?0?$AA?5@ 10006080     swiusb.obj
 0002:00001100       ??_C@_1HK@CKAODNBP@?$AA?$CF?$AAs?$AA?5?$AAE?$AAr?$AAr?$AAo?$AAr?$AA?5?$AAt?$AAo?$AA?5?$AAr?$AAe?$AAa?$AAd?$AA?5?$AA?$CF?$AAd?$AA?5?$AAb?$AAy?$AAt?$AAe?$AAs?$AA?5?$AAf?$AAr?$AAo?$AAm?$AA?5?$AA?$CF@ 10006100     swiusb.obj
 0002:00001180       ??_C@_1EK@LFOGABOB@?$AA?$CF?$AAs?$AA?5?$AAF?$AAi?$AAn?$AAi?$AAs?$AAh?$AA?5?$AAd?$AAo?$AAw?$AAn?$AAl?$AAo?$AAa?$AAd?$AAi?$AAn?$AAg?$AA?5?$AA?$CF?$AAs?$AA?0?$AA?5?$AAt?$AAc?$AA?5?$AA?$DN?$AA?5?$AA?$CF@ 10006180     swiusb.obj
 0002:000011d0       ??_C@_1GE@DCHBGCNO@?$AA?$CF?$AAs?$AA?5?$AAB?$AAy?$AAt?$AAe?$AAs?$AA?5?$AAt?$AAo?$AA?5?$AAs?$AAe?$AAn?$AAd?$AA?5?$AAi?$AAs?$AA?5?$AA5?$AA1?$AA2?$AA?5?$AAb?$AAy?$AAt?$AAe?$AAs?$AA?0?$AA?5?$AAf@ 100061d0     swiusb.obj
 0002:00001234       ??_C@_1CC@KMPLKPBO@?$AAS?$AAW?$AAI?$AAQ?$AAD?$AAL?$AA?5?$AAS?$AAe?$AAn?$AAd?$AAD?$AAa?$AAt?$AAa?$AA?3?$AA?$AA@ 10006234     swiusb.obj
 0002:00001258       ??_C@_1EI@FNKDFGHM@?$AA?$CF?$AAs?$AA?5?$AAS?$AAt?$AAa?$AAr?$AAt?$AA?5?$AAd?$AAo?$AAw?$AAn?$AAl?$AAo?$AAa?$AAd?$AAi?$AAn?$AAg?$AA?5?$AA?$CF?$AAs?$AA?0?$AA?5?$AAt?$AAc?$AA?5?$AA?$DN?$AA?5?$AA?$CF?$AAd@ 10006258     swiusb.obj
 0002:000012a0       ??_C@_0BN@NLFGIBBM@QCOM?5high?5speed?5protocol?5hst?$AA@ 100062a0     swiusb.obj
 0002:000012c0       ??_C@_1GI@DIJPPCPI@?$AA?$CF?$AAs?$AA?5?$AAS?$AAt?$AAa?$AAt?$AAe?$AA?5?$AAm?$AAa?$AAc?$AAh?$AAi?$AAn?$AAe?$AA?5?$AAe?$AAx?$AAi?$AAt?$AAs?$AA?5?$AAd?$AAu?$AAe?$AA?5?$AAt?$AAo?$AA?5?$AAt?$AAh@ 100062c0     swiusb.obj
 0002:00001328       ??_C@_1DG@FDGDPEEN@?$AAS?$AAW?$AAI?$AAQ?$AAD?$AAL?$AA?5?$AAS?$AAt?$AAa?$AAt?$AAe?$AAM?$AAa?$AAc?$AAh?$AAi?$AAn?$AAe?$AAT?$AAh?$AAr?$AAe?$AAa?$AAd?$AA?3?$AA?$AA@ 10006328     swiusb.obj
 0002:00001360       ??_C@_1EG@DEIIKEDH@?$AA?$CF?$AAs?$AA?5?$AAS?$AAi?$AAg?$AAn?$AAa?$AAl?$AA?5?$AAs?$AAh?$AAu?$AAt?$AA?5?$AAd?$AAo?$AAw?$AAn?$AA?5?$AAm?$AAo?$AAd?$AAe?$AAm?$AA?5?$AAe?$AAv?$AAe?$AAn?$AAt?$AA?4@ 10006360     swiusb.obj
 0002:000013a8       ??_C@_1CO@DOCJGIKP@?$AA?$CF?$AAs?$AA?5?$AA?$CF?$AAs?$AA?5?$AAf?$AAi?$AAl?$AAe?$AA?5?$AAs?$AAi?$AAz?$AAe?$AA?3?$AA?5?$AA?$CF?$AAd?$AA?4?$AA?$AN?$AA?6?$AA?$AA@ 100063a8     swiusb.obj
 0002:000013d8       ??_C@_1CE@JGKGKFDL@?$AAS?$AAW?$AAI?$AAQ?$AAD?$AAL?$AA?5?$AAG?$AAe?$AAt?$AAF?$AAW?$AAF?$AAi?$AAl?$AAe?$AA?3?$AA?$AA@ 100063d8     swiusb.obj
 0002:00001400       ??_C@_1FE@LDIAPPKN@?$AA?$CF?$AAs?$AA?5?$AAF?$AAa?$AAi?$AAl?$AAe?$AAd?$AA?5?$AAt?$AAo?$AA?5?$AAr?$AAe?$AAt?$AAr?$AAi?$AAe?$AAv?$AAe?$AA?5?$AAf?$AAi?$AAl?$AAe?$AA?5?$AAs?$AAi?$AAz?$AAe?$AA?5@ 10006400     swiusb.obj
 0002:00001458       ??_C@_1EA@PCODGBJO@?$AA?$CF?$AAs?$AA?5?$AAF?$AAa?$AAi?$AAl?$AAe?$AAd?$AA?5?$AAt?$AAo?$AA?5?$AAo?$AAp?$AAe?$AAn?$AA?5?$AAu?$AAq?$AAc?$AAn?$AA?5?$AAa?$AAt?$AA?5?$AA?$CF?$AAs?$AA?4?$AA?$AN?$AA?6?$AA?$AA@ 10006458     swiusb.obj
 0002:00001498       ??_C@_1EA@HEDOKPDJ@?$AA?$CF?$AAs?$AA?5?$AAF?$AAa?$AAi?$AAl?$AAe?$AAd?$AA?5?$AAt?$AAo?$AA?5?$AAo?$AAp?$AAe?$AAn?$AA?5?$AAa?$AAp?$AAp?$AAs?$AA?5?$AAa?$AAt?$AA?5?$AA?$CF?$AAs?$AA?4?$AA?$AN?$AA?6?$AA?$AA@ 10006498     swiusb.obj
 0002:000014d8       ??_C@_1EA@BONCEAJM@?$AA?$CF?$AAs?$AA?5?$AAF?$AAa?$AAi?$AAl?$AAe?$AAd?$AA?5?$AAt?$AAo?$AA?5?$AAo?$AAp?$AAe?$AAn?$AA?5?$AAa?$AAm?$AAs?$AAs?$AA?5?$AAa?$AAt?$AA?5?$AA?$CF?$AAs?$AA?4?$AA?$AN?$AA?6?$AA?$AA@ 100064d8     swiusb.obj
 0002:00001518       ??_C@_1BC@GLIGFLDD@?$AA?$CF?$AAs?$AA?2?$AA?$CF?$AAs?$AA?2?$AA?$CF?$AAs?$AA?$AA@ 10006518     swiusb.obj
 0002:0000152c       ??_C@_13LPLIHJO@?$AA6?$AA?$AA@ 1000652c     swiusb.obj
 0002:00001530       ??_C@_19LPHHOHBE@?$AAU?$AAM?$AAT?$AAS?$AA?$AA@ 10006530     swiusb.obj
 0002:0000153c       ??_C@_1BC@OFAJFMNA@?$AA?$CF?$AAs?$AA?2?$AA?$CF?$AAs?$AA_?$AA?$CF?$AAs?$AA?$AA@ 1000653c     swiusb.obj
 0002:00001550       ??_C@_1BC@KOPEMBKC@?$AA?$CF?$AAs?$AA?2?$AA?$CF?$AAd?$AA?2?$AA?$CF?$AAs?$AA?$AA@ 10006550     swiusb.obj
 0002:00001564       ??_C@_1BC@HBBIFKBJ@?$AAu?$AAq?$AAc?$AAn?$AA?4?$AAm?$AAb?$AAn?$AA?$AA@ 10006564     swiusb.obj
 0002:00001578       ??_C@_1BC@HCBPLFDD@?$AAa?$AAp?$AAp?$AAs?$AA?4?$AAm?$AAb?$AAn?$AA?$AA@ 10006578     swiusb.obj
 0002:0000158c       ??_C@_1BC@OBBDOMCP@?$AAa?$AAm?$AAs?$AAs?$AA?4?$AAm?$AAb?$AAn?$AA?$AA@ 1000658c     swiusb.obj
 0002:000015a0       ??_C@_1BC@CAHLMGEB@?$AA?$CF?$AAs?$AA?2?$AA?$CF?$AAd?$AA_?$AA?$CF?$AAs?$AA?$AA@ 100065a0     swiusb.obj
 0002:000015b8       ??_C@_1FE@FIJDOLFA@?$AA?$CF?$AAs?$AA?5?$AAG?$AAo?$AAb?$AAi?$AA?5?$AAf?$AAi?$AAr?$AAm?$AAw?$AAa?$AAr?$AAe?$AA?5?$AAl?$AAo?$AAc?$AAa?$AAt?$AAi?$AAo?$AAn?$AA?5?$AAi?$AAn?$AAf?$AAo?$AA?5?$AAm@ 100065b8     swiusb.obj
 0002:00001610       ??_C@_1GK@GDHMCFNB@?$AA?$CF?$AAs?$AA?5?$AAF?$AAa?$AAi?$AAl?$AAe?$AAd?$AA?5?$AAt?$AAo?$AA?5?$AAr?$AAe?$AAa?$AAd?$AA?5?$AAc?$AAa?$AAr?$AAr?$AAi?$AAe?$AAr?$AA?5?$AAi?$AAn?$AAd?$AAe?$AAx?$AA?5@ 10006610     swiusb.obj
 0002:0000167c       ??_C@_1BK@GIONEDDC@?$AAC?$AAa?$AAr?$AAr?$AAi?$AAe?$AAr?$AAI?$AAn?$AAd?$AAe?$AAx?$AA?$AA@ 1000667c     swiusb.obj
 0002:00001698       ??_C@_1BC@GPCOMFMF@?$AA?2?$AAw?$AAi?$AAn?$AAd?$AAo?$AAw?$AAs?$AA?$AA@ 10006698     swiusb.obj
 0002:000016ac       ??_C@_1DA@GOOEJGGD@?$AAS?$AAW?$AAI?$AAQ?$AAD?$AAL?$AA?5?$AAG?$AAe?$AAt?$AAG?$AAo?$AAb?$AAi?$AAF?$AAi?$AAr?$AAm?$AAw?$AAa?$AAr?$AAe?$AA?3?$AA?$AA@ 100066ac     swiusb.obj
 0002:000016e0       ??_C@_1GG@BJFBPNCJ@?$AA?$CF?$AAs?$AA?5?$AAF?$AAa?$AAi?$AAl?$AAe?$AAd?$AA?5?$AAt?$AAo?$AA?5?$AAr?$AAe?$AAa?$AAd?$AA?5?$AAf?$AAw?$AA?5?$AAl?$AAo?$AAc?$AAa?$AAt?$AAi?$AAo?$AAn?$AA?5?$AAf?$AAr@ 100066e0     swiusb.obj
 0002:00001748       ??_C@_1CC@OPPLHLDH@?$AAF?$AAi?$AAr?$AAm?$AAw?$AAa?$AAr?$AAe?$AAL?$AAo?$AAc?$AAa?$AAt?$AAi?$AAo?$AAn?$AA?$AA@ 10006748     swiusb.obj
 0002:00001770       ??_C@_1EG@OCNEBEOA@?$AA?2?$AAS?$AAo?$AAf?$AAt?$AAw?$AAa?$AAr?$AAe?$AA?2?$AAS?$AAi?$AAe?$AAr?$AAr?$AAa?$AA?5?$AAW?$AAi?$AAr?$AAe?$AAl?$AAe?$AAs?$AAs?$AA?5?$AAI?$AAn?$AAc?$AA?2?$AAQ?$AAD@ 10006770     swiusb.obj
 0002:000017b8       ??_C@_1DO@KFEBCBMK@?$AAS?$AAW?$AAI?$AAQ?$AAD?$AAL?$AA?5?$AAP?$AAa?$AAr?$AAs?$AAe?$AAA?$AAn?$AAd?$AAA?$AAd?$AAd?$AAT?$AAo?$AAR?$AAe?$AAa?$AAd?$AAQ?$AAu?$AAe?$AAu?$AAe?$AA?3?$AA?$AA@ 100067b8     swiusb.obj
 0002:000017f8       ??_C@_1GK@GKBHNADO@?$AA?$CF?$AAs?$AA?5?$AAF?$AAr?$AAa?$AAm?$AAe?$AA?5?$AAh?$AAe?$AAa?$AAd?$AAe?$AAr?$AA?5?$AAi?$AAs?$AA?5?$AAm?$AAi?$AAs?$AAs?$AAi?$AAn?$AAg?$AA?5?$AAi?$AAn?$AA?5?$AAt?$AAh@ 100067f8     swiusb.obj
 0002:00001868       ??_C@_1FA@IMPGNDBA@?$AA?6?$AA?$CF?$AAs?$AA?5?$AAC?$AAh?$AAa?$AAn?$AAn?$AAe?$AAl?$AA?5?$AA?$CD?$AA?$CF?$AAd?$AA?5?$AAe?$AAx?$AAi?$AAt?$AAs?$AA?0?$AA?5?$AAt?$AAi?$AAc?$AAk?$AAC?$AAo?$AAu?$AAn?$AAt@ 10006868     swiusb.obj
 0002:000018b8       ??_C@_1FG@FMCBPJCB@?$AA?$CF?$AAs?$AA?5?$AAC?$AAh?$AAa?$AAn?$AAn?$AAe?$AAl?$AA?5?$AA?$CD?$AA?$CF?$AAd?$AA?5?$AAe?$AAx?$AAi?$AAt?$AAs?$AA?5?$AAb?$AAc?$AAo?$AAs?$AA?5?$AAU?$AAS?$AAB?$AA?5?$AAD?$AAe@ 100068b8     swiusb.obj
 0002:00001910       ??_C@_1FM@MOJPBCHF@?$AA?$CF?$AAs?$AA?5?$AAC?$AAl?$AAo?$AAs?$AAe?$AA?5?$AAt?$AAr?$AAa?$AAn?$AAs?$AAf?$AAe?$AAr?$AA?5?$AAf?$AAa?$AAi?$AAl?$AAe?$AAd?$AA?5?$AAi?$AAn?$AA?5?$AAb?$AAu?$AAl?$AAk@ 10006910     swiusb.obj
 0002:00001970       ??_C@_1IG@BJEMNGMM@?$AA?$CF?$AAs?$AA?5?$AAA?$AAb?$AAo?$AAr?$AAt?$AA?5?$AAt?$AAr?$AAa?$AAn?$AAs?$AAf?$AAe?$AAr?$AA?5?$AAr?$AAe?$AAt?$AAu?$AAr?$AAn?$AAs?$AA?5?$AAe?$AAr?$AAr?$AAo?$AAr?$AA?5@ 10006970     swiusb.obj
 0002:000019f8       ??_C@_1GC@NDPAIODL@?$AA?$CF?$AAs?$AA?5?$AAT?$AAr?$AAa?$AAn?$AAs?$AAf?$AAe?$AAr?$AA?5?$AAc?$AAo?$AAm?$AAp?$AAl?$AAe?$AAt?$AAe?$AA?5?$AAf?$AAa?$AAi?$AAl?$AAe?$AAd?$AA?5?$AAi?$AAn?$AA?5?$AAb@ 100069f8     swiusb.obj
 0002:00001a60       ??_C@_1IA@IMIFELAB@?$AA?$CF?$AAs?$AA?5?$AAG?$AAe?$AAt?$AA?5?$AAt?$AAr?$AAa?$AAn?$AAs?$AAf?$AAe?$AAr?$AA?5?$AAs?$AAt?$AAa?$AAt?$AAu?$AAs?$AA?5?$AAe?$AAr?$AAr?$AAo?$AAr?$AA?5?$AAi?$AAn?$AA?5@ 10006a60     swiusb.obj
 0002:00001ae0       ??_C@_1FK@BLDOOIEH@?$AAS?$AAW?$AAI?$AAQ?$AAD?$AAL?$AA?3?$AA?5?$AAR?$AAX?$AA?5?$AAD?$AAA?$AAT?$AAA?$AA?5?$AA?9?$AA?5?$AAB?$AAu?$AAl?$AAk?$AAI?$AAn?$AAT?$AAh?$AAr?$AAe?$AAa?$AAd?$AA?3?$AA?5@ 10006ae0     swiusb.obj
 0002:00001b3c       ??_C@_1CK@EPBNGFEH@?$AAS?$AAW?$AAI?$AAQ?$AAD?$AAL?$AA?5?$AAB?$AAu?$AAl?$AAk?$AAI?$AAn?$AAT?$AAh?$AAr?$AAe?$AAa?$AAd?$AA?3?$AA?$AA@ 10006b3c     swiusb.obj
 0002:00001b68       ??_C@_1HG@HMHKLKGM@?$AA?$CF?$AAs?$AA?5?$AAF?$AAa?$AAi?$AAl?$AAe?$AAd?$AA?5?$AAt?$AAo?$AA?5?$AAa?$AAl?$AAl?$AAo?$AAc?$AAa?$AAt?$AAe?$AA?5?$AAr?$AAe?$AAc?$AAe?$AAi?$AAv?$AAe?$AA?5?$AAb?$AAu@ 10006b68     swiusb.obj
 0002:00001be0       ??_C@_1DI@MFGINILI@?$AA?$AN?$AA?6?$AAB?$AAu?$AAl?$AAk?$AAI?$AAn?$AAT?$AAh?$AAr?$AAe?$AAa?$AAd?$AA?0?$AA?5?$AAC?$AAh?$AAa?$AAn?$AAn?$AAe?$AAl?$AA?5?$AA?$CD?$AA?$CF?$AAd?$AA?$AA@ 10006be0     swiusb.obj
 0002:00001c18       ??_C@_1BG@EAJJPHIA@?$AA?$CF?$AAs?$AA?5?$AAD?$AAo?$AAn?$AAe?$AA?4?$AA?$AN?$AA?6?$AA?$AA@ 10006c18     swiusb.obj
 0002:00001c30       ??_C@_1FI@OPEIDNFI@?$AA?$CF?$AAs?$AA?5?$AAF?$AAa?$AAi?$AAl?$AAe?$AAd?$AA?5?$AAt?$AAo?$AA?5?$AAc?$AAr?$AAe?$AAa?$AAt?$AAe?$AA?5?$AAs?$AAt?$AAa?$AAt?$AAe?$AA?5?$AAm?$AAa?$AAc?$AAh?$AAi?$AAn@ 10006c30     swiusb.obj
 0002:00001c88       ??_C@_1FE@CDBFECJ@?$AA?$CF?$AAs?$AA?5?$AAF?$AAa?$AAi?$AAl?$AAe?$AAd?$AA?5?$AAt?$AAo?$AA?5?$AAc?$AAr?$AAe?$AAa?$AAt?$AAe?$AA?5?$AAs?$AAt?$AAa?$AAt?$AAe?$AA?5?$AAc?$AAh?$AAa?$AAn?$AAg?$AAe@ 10006c88     swiusb.obj
 0002:00001ce0       ??_C@_1FC@HFCHPNJM@?$AA?$CF?$AAs?$AA?5?$AAM?$AAi?$AAs?$AAs?$AA?5?$AAC?$AAo?$AAn?$AAf?$AAi?$AAg?$AAu?$AAr?$AAa?$AAt?$AAi?$AAo?$AAn?$AA?5?$AAD?$AAe?$AAs?$AAc?$AAr?$AAi?$AAp?$AAt?$AAo?$AAr@ 10006ce0     swiusb.obj
 0002:00001d38       ??_C@_1FG@LCIGEFBO@?$AA?$CF?$AAs?$AA?5?$AAB?$AAu?$AAl?$AAk?$AAo?$AAu?$AAt?$AA?5?$AAt?$AAh?$AAr?$AAe?$AAa?$AAd?$AA?5?$AAp?$AAr?$AAi?$AAo?$AAr?$AAi?$AAt?$AAy?$AA?5?$AAi?$AAs?$AA?5?$AAs?$AAe@ 10006d38     swiusb.obj
 0002:00001d90       ??_C@_1HC@EJJGKLHO@?$AA?$CF?$AAs?$AA?5?$AAF?$AAa?$AAi?$AAl?$AAe?$AAd?$AA?5?$AAt?$AAo?$AA?5?$AAs?$AAe?$AAt?$AA?5?$AAt?$AAh?$AAr?$AAe?$AAa?$AAd?$AA?5?$AAp?$AAr?$AAi?$AAo?$AAr?$AAi?$AAt?$AAy@ 10006d90     swiusb.obj
 0002:00001e08       ??_C@_1FE@KJFMHGDO@?$AA?$CF?$AAs?$AA?5?$AAB?$AAu?$AAl?$AAk?$AAi?$AAn?$AA?5?$AAt?$AAh?$AAr?$AAe?$AAa?$AAd?$AA?5?$AAp?$AAr?$AAi?$AAo?$AAr?$AAi?$AAt?$AAy?$AA?5?$AAi?$AAs?$AA?5?$AAs?$AAe?$AAt@ 10006e08     swiusb.obj
 0002:00001e60       ??_C@_1HA@BFPHAFJG@?$AA?$CF?$AAs?$AA?5?$AAF?$AAa?$AAi?$AAl?$AAe?$AAd?$AA?5?$AAt?$AAo?$AA?5?$AAs?$AAe?$AAt?$AA?5?$AAt?$AAh?$AAr?$AAe?$AAa?$AAd?$AA?5?$AAp?$AAr?$AAi?$AAo?$AAr?$AAi?$AAt?$AAy@ 10006e60     swiusb.obj
 0002:00001ed0       ??_C@_1HC@POHDHBIF@?$AA?$CF?$AAs?$AA?5?$AAF?$AAa?$AAi?$AAl?$AAe?$AAd?$AA?5?$AAt?$AAo?$AA?5?$AAr?$AAe?$AAs?$AAe?$AAr?$AAv?$AAe?$AA?5?$AAa?$AAn?$AAd?$AA?5?$AAc?$AAo?$AAm?$AAm?$AAi?$AAt?$AA?5@ 10006ed0     swiusb.obj
 0002:00001f48       ??_C@_1FI@FNFGEIJL@?$AA?$CF?$AAs?$AA?5?$AAC?$AAo?$AAm?$AAm?$AAi?$AAt?$AAt?$AAe?$AAd?$AA?5?$AAm?$AAe?$AAm?$AAo?$AAr?$AAy?$AA?5?$AAf?$AAo?$AAr?$AA?5?$AAo?$AAu?$AAt?$AA?5?$AAb?$AAu?$AAf?$AAf@ 10006f48     swiusb.obj
 0002:00001fa0       ??_C@_1GC@KFGFIALK@?$AA?$CF?$AAs?$AA?5?$AAF?$AAa?$AAi?$AAl?$AAe?$AAd?$AA?5?$AAt?$AAo?$AA?5?$AAa?$AAl?$AAl?$AAo?$AAc?$AAa?$AAt?$AAe?$AA?5?$AAm?$AAe?$AAm?$AAo?$AAr?$AAy?$AA?5?$AAf?$AAo?$AAr@ 10006fa0     swiusb.obj
 0002:00002004       ??_C@_1DI@OMOADICB@?$AA?$CF?$AAs?$AA?5?$AAE?$AAr?$AAr?$AAo?$AAr?$AA?5?$AAi?$AAn?$AA?5?$AAG?$AAe?$AAt?$AAD?$AAe?$AAv?$AAi?$AAc?$AAe?$AAI?$AAn?$AAf?$AAo?$AA?$AN?$AA?6?$AA?$AA@ 10007004     swiusb.obj
 0002:00002040       ??_C@_1EO@HEBGAPDJ@?$AA?$CF?$AAs?$AA?5?$AAR?$AAe?$AAt?$AAu?$AAr?$AAn?$AAs?$AA?5?$AAA?$AAc?$AAc?$AAe?$AAp?$AAt?$AAC?$AAo?$AAn?$AAt?$AAr?$AAo?$AAl?$AA?5?$AAr?$AAi?$AAg?$AAh?$AAt?$AA?5?$AAa@ 10007040     swiusb.obj
 0002:00002090       ??_C@_1EI@EPHLGOBO@?$AA?$CF?$AAs?$AA?5?$AAF?$AAa?$AAi?$AAl?$AAe?$AAd?$AA?5?$AAt?$AAo?$AA?5?$AAc?$AAr?$AAe?$AAa?$AAt?$AAe?$AA?5?$AAS?$AAW?$AAI?$AAQ?$AAD?$AAL?$AA_?$AAE?$AAV?$AAE?$AAN?$AAT@ 10007090     swiusb.obj
 0002:000020d8       ??_C@_1BK@DFHDIHFD@?$AAS?$AAW?$AAI?$AAQ?$AAD?$AAL?$AA_?$AAE?$AAV?$AAE?$AAN?$AAT?$AA?$AA@ 100070d8     swiusb.obj
 0002:000020f8       ??_C@_1HK@OGFFKEKI@?$AA?$CF?$AAs?$AA?5?$AAF?$AAa?$AAi?$AAl?$AAe?$AAd?$AA?5?$AAb?$AAe?$AAc?$AAa?$AAu?$AAs?$AAe?$AA?5?$AAp?$AAr?$AAe?$AAv?$AAi?$AAo?$AAu?$AAs?$AA?5?$AAd?$AAr?$AAi?$AAv?$AAe@ 100070f8     swiusb.obj
 0002:00002178       ??_C@_1GK@FPCDCMGN@?$AA?$CF?$AAs?$AA?5?$AAF?$AAa?$AAi?$AAl?$AAe?$AAd?$AA?5?$AAt?$AAo?$AA?5?$AAc?$AAr?$AAe?$AAa?$AAt?$AAe?$AA?5?$AAm?$AAo?$AAd?$AAe?$AAm?$AA?5?$AAs?$AAh?$AAu?$AAt?$AA?5?$AAd@ 10007178     swiusb.obj
 0002:000021e8       ??_C@_1GE@PCKLIPAE@?$AA?$CF?$AAs?$AA?5?$AAF?$AAa?$AAi?$AAl?$AAe?$AAd?$AA?5?$AAt?$AAo?$AA?5?$AAc?$AAr?$AAe?$AAa?$AAt?$AAe?$AA?5?$AAm?$AAo?$AAd?$AAe?$AAm?$AA_?$AAn?$AAe?$AAe?$AAd?$AAs?$AA_@ 100071e8     swiusb.obj
 0002:0000224c       ??_C@_1DC@HOGOPNOP@?$AAS?$AAW?$AAI?$AA_?$AAm?$AAo?$AAd?$AAe?$AAm?$AA_?$AAn?$AAe?$AAe?$AAd?$AAs?$AA_?$AAs?$AAh?$AAu?$AAt?$AAd?$AAo?$AAw?$AAn?$AA?$AA@ 1000724c     swiusb.obj
 0002:00002280       ??_C@_1CC@CGONKFLE@?$AAI?$AAn?$AAT?$AAh?$AAr?$AAe?$AAa?$AAd?$AAP?$AAr?$AAi?$AAo?$AAr?$AAi?$AAt?$AAy?$AA?$AA@ 10007280     swiusb.obj
 0002:000022a4       ??_C@_1CE@NHOFNKJK@?$AAO?$AAu?$AAt?$AAT?$AAh?$AAr?$AAe?$AAa?$AAd?$AAP?$AAr?$AAi?$AAo?$AAr?$AAi?$AAt?$AAy?$AA?$AA@ 100072a4     swiusb.obj
 0002:000022c8       ??_C@_1BM@JHKEMJFJ@?$AAF?$AAa?$AAi?$AAl?$AAu?$AAr?$AAe?$AAP?$AAr?$AAo?$AAm?$AAp?$AAt?$AA?$AA@ 100072c8     swiusb.obj
 0002:000022e8       ??_C@_1FM@GNKFILCP@?$AA?$CF?$AAs?$AA?5?$AAM?$AAa?$AAx?$AAi?$AAm?$AAu?$AAm?$AA?5?$AAr?$AAe?$AAt?$AAr?$AAy?$AA?5?$AAs?$AAe?$AAt?$AAt?$AAi?$AAn?$AAg?$AA?5?$AAf?$AAr?$AAo?$AAm?$AA?5?$AAr?$AAe@ 100072e8     swiusb.obj
 0002:00002344       ??_C@_1DA@GGPODMLA@?$AAS?$AAW?$AAI?$AAQ?$AAD?$AAL?$AA?5?$AAU?$AAS?$AAB?$AAD?$AAe?$AAv?$AAi?$AAc?$AAe?$AAA?$AAt?$AAt?$AAa?$AAc?$AAh?$AA?3?$AA?$AA@ 10007344     swiusb.obj
 0002:00002378       ??_C@_1HM@MMKHCDKK@?$AA?$CF?$AAs?$AA?5?$AAM?$AAa?$AAx?$AAi?$AAm?$AAu?$AAm?$AA?5?$AAr?$AAe?$AAt?$AAr?$AAi?$AAe?$AAs?$AA?5?$AAu?$AAn?$AAs?$AAp?$AAe?$AAc?$AAi?$AAf?$AAi?$AAe?$AAd?$AA?0?$AA?5@ 10007378     swiusb.obj
 0002:000023f4       ??_C@_1BO@ELNPIGOJ@?$AAM?$AAa?$AAx?$AAi?$AAm?$AAu?$AAm?$AAR?$AAe?$AAt?$AAr?$AAi?$AAe?$AAs?$AA?$AA@ 100073f4     swiusb.obj
 0002:00002414       ??_C@_0L@FFLPPCPC@2?43?40?4248?$AA?$AA@ 10007414     swiusb.obj
 0002:00002420       ??_C@_1GO@DBDMICLH@?$AAS?$AAW?$AAI?$AAQ?$AAD?$AAL?$AA?5?$AA?$CF?$AAs?$AA?5?$AA?9?$AA?5?$AAU?$AAS?$AAB?$AAD?$AAe?$AAv?$AAi?$AAc?$AAe?$AAA?$AAt?$AAt?$AAa?$AAc?$AAh?$AA?$CI?$AA?$CJ?$AA?5?$AAc?$AAa@ 10007420     swiusb.obj
 0002:0000249c       __IMPORT_DESCRIPTOR_COREDLL 1000749c     coredll:COREDLL.dll
 0002:000024b0       __NULL_IMPORT_DESCRIPTOR   100074b0     coredll:COREDLL.dll
 0003:00000000       __imp_EventModify          10008000     coredll:COREDLL.dll
 0003:00000004       __imp_NKDbgPrintfW         10008004     coredll:COREDLL.dll
 0003:00000008       __imp_GlobalMemoryStatus   10008008     coredll:COREDLL.dll
 0003:0000000c       __imp_GetLastError         1000800c     coredll:COREDLL.dll
 0003:00000010       __imp_WaitForMultipleObjects 10008010     coredll:COREDLL.dll
 0003:00000014       __imp_GetTickCount         10008014     coredll:COREDLL.dll
 0003:00000018       __imp_WaitForSingleObject  10008018     coredll:COREDLL.dll
 0003:0000001c       __imp___rt_udiv            1000801c     coredll:COREDLL.dll
 0003:00000020       __imp_LocalFree            10008020     coredll:COREDLL.dll
 0003:00000024       __imp_VirtualFree          10008024     coredll:COREDLL.dll
 0003:00000028       __imp_TerminateThread      10008028     coredll:COREDLL.dll
 0003:0000002c       __imp_CloseHandle          1000802c     coredll:COREDLL.dll
 0003:00000030       __imp_Sleep                10008030     coredll:COREDLL.dll
 0003:00000034       __imp_ReadFile             10008034     coredll:COREDLL.dll
 0003:00000038       __imp_SetFilePointer       10008038     coredll:COREDLL.dll
 0003:0000003c       __imp_memcpy               1000803c     coredll:COREDLL.dll
 0003:00000040       __imp_memset               10008040     coredll:COREDLL.dll
 0003:00000044       __imp_GetFileSize          10008044     coredll:COREDLL.dll
 0003:00000048       __imp_CreateFileW          10008048     coredll:COREDLL.dll
 0003:0000004c       __imp_swprintf             1000804c     coredll:COREDLL.dll
 0003:00000050       __imp_RegCloseKey          10008050     coredll:COREDLL.dll
 0003:00000054       __imp__wcslwr              10008054     coredll:COREDLL.dll
 0003:00000058       __imp_RegQueryValueExW     10008058     coredll:COREDLL.dll
 0003:0000005c       __imp_RegOpenKeyExW        1000805c     coredll:COREDLL.dll
 0003:00000060       __imp_wcscmp               10008060     coredll:COREDLL.dll
 0003:00000064       __imp_VirtualAlloc         10008064     coredll:COREDLL.dll
 0003:00000068       __imp_CeSetThreadPriority  10008068     coredll:COREDLL.dll
 0003:0000006c       __imp_CreateThread         1000806c     coredll:COREDLL.dll
 0003:00000070       __imp_LocalAlloc           10008070     coredll:COREDLL.dll
 0003:00000074       __imp_CreateEventW         10008074     coredll:COREDLL.dll
 0003:00000078       __imp_MultiByteToWideChar  10008078     coredll:COREDLL.dll
 0003:0000007c       __imp___report_gsfailure   1000807c     coredll:COREDLL.dll
 0003:00000080       __imp_DisableThreadLibraryCalls 10008080     coredll:COREDLL.dll
 0003:00000084       __imp___security_gen_cookie 10008084     coredll:COREDLL.dll
 0003:00000088       \177COREDLL_NULL_THUNK_DATA 10008088     coredll:COREDLL.dll
 0003:0000008c       __xc_a                     1000808c     corelibc:crt0init.obj
 0003:00000094       __xc_z                     10008094     corelibc:crt0init.obj
 0003:00000098       __xi_a                     10008098     corelibc:crt0init.obj
 0003:0000009c       __xi_z                     1000809c     corelibc:crt0init.obj
 0003:000000a0       __xp_a                     100080a0     corelibc:crt0init.obj
 0003:000000a4       __xp_z                     100080a4     corelibc:crt0init.obj
 0003:000000a8       __xt_a                     100080a8     corelibc:crt0init.obj
 0003:000000ac       __xt_z                     100080ac     corelibc:crt0init.obj
 0003:000002b0       ?fFWFolder@@3HA            100082b0     swiusb.obj
 0003:000002b4       ?gdwMaxRetries@@3KA        100082b4     swiusb.obj
 0003:000002b8       __security_cookie_complement 100082b8     corelibc:seccook.obj
 0003:000002bc       __security_cookie          100082bc     corelibc:seccook.obj
 0003:000002c0       ?ghDeviceInstalledEvent@@3PAXA 100082c0     swiusb.obj
 0003:000002c4       ?hDeviceCloseEvent@@3PAXA  100082c4     swiusb.obj
 0003:000002c8       ?hAbortEvent@@3PAXA        100082c8     swiusb.obj
 0003:000002cc       ?ghQDLEvent@@3PAXA         100082cc     swiusb.obj
 0003:000002d0       ?ghShutDownEvent@@3PAXA    100082d0     swiusb.obj
 0003:000002d4       ?ghShutDownRequestEvent@@3PAXA 100082d4     swiusb.obj
 0003:000002d8       ?gfGobi3k@@3HA             100082d8     swiusb.obj
 0003:000002dc       ?gdwRetries@@3KA           100082dc     swiusb.obj
 0003:000002e0       ?gModem@@3U_SW_MODEM@@A    100082e0     swiusb.obj
 0003:00000614       __onexitend                10008614     <common>
 0003:00000618       __onexitbegin              10008618     <common>
 0003:0000061c       _exitflag                  1000861c     <common>
 0003:00000620       _pRawDllMain               10008620     <common>

 entry point at        0001:000034a4

 Static symbols

 0001:00000210       ?TransmitBytes@@YAHPAU_SW_CHANNEL@@PAEI@Z 10001210 f   swiusb.obj
 0001:00003600       doexit                     10004600 f   corelibc:crt0dat.obj

 Exports

  ordinal    name

        1    USBDeviceAttach
        2    USBInstallDriver
